 esai_wm8580

 Timestamp is 4da293c0 (Mon Apr 11 17:38:08 2011)

 Preferred load address is 10000000

 Start         Length     Name                   Class
 0001:00000000 00000910H .rdata                  CODE
 0001:00000910 00000028H .rdata$debug            CODE
 0001:00000938 00007388H .text                   CODE
 0001:00007cc0 0000003cH .xdata                  CODE
 0001:00007cfc 00000064H .idata$2                CODE
 0001:00007d60 00000014H .idata$3                CODE
 0001:00007d74 000000f8H .idata$4                CODE
 0001:00007e6c 00000188H .idata$6                CODE
 0001:00008000 0000009bH .edata                  CODE
 0002:00000000 000000f8H .idata$5                DATA
 0002:000000f8 00000018H .data                   DATA
 0002:00000110 00000020H .bss                    DATA
 0003:00000000 00000898H .pdata                  DATA

  Address         Publics by Value              Rva+Base       Lib:Object

 0000:00000000       ___safe_se_handler_count   00000000     <absolute>
 0000:00000000       ___safe_se_handler_table   00000000     <absolute>
 0001:0000001c       ??_C@_1M@BALJCCCP@?$AAS?$AAP?$AAI?$AA1?$AA?3?$AA?$AA@ 1000101c     wm8580.obj
 0001:00000028       ??_C@_1M@LCEEOPDH@?$AAI?$AA2?$AAC?$AA1?$AA?3?$AA?$AA@ 10001028     ak5702.obj
 0001:000000f8       ??_7InputDeviceContext@@6B@ 100010f8     esai_common_topaz_v1:hwctxt.obj
 0001:00000120       ??_7OutputDeviceContext@@6B@ 10001120     esai_common_topaz_v1:hwctxt.obj
 0001:00000148       ??_C@_1BI@BHLBGEOK@?$AAP?$AAr?$AAi?$AAo?$AAr?$AAi?$AAt?$AAy?$AA2?$AA5?$AA6?$AA?$AA@ 10001148     esai_common_topaz_v1:hwctxt.obj
 0001:00000160       ??_7DeviceContext@@6B@     10001160     esai_common_topaz_v1:devctxt.obj
 0001:00000260       ??_7OutputStreamContextEx@@6B@ 10001260     esai_common_topaz_v1:devctxt.obj
 0001:000002a8       ??_7OutputStreamContextM8@@6B@ 100012a8     esai_common_topaz_v1:devctxt.obj
 0001:000002f0       ??_7OutputStreamContextS8@@6B@ 100012f0     esai_common_topaz_v1:devctxt.obj
 0001:00000338       ??_7OutputStreamContextM16@@6B@ 10001338     esai_common_topaz_v1:devctxt.obj
 0001:00000380       ??_7OutputStreamContextS16@@6B@ 10001380     esai_common_topaz_v1:devctxt.obj
 0001:000003c8       ??_7InputStreamContextEx@@6B@ 100013c8     esai_common_topaz_v1:devctxt.obj
 0001:000005a0       ??_7StreamContext@@6B@     100015a0     esai_common_topaz_v1:strmctxt.obj
 0001:000005dc       ??_C@_1BC@JBIMOOCB@?$AAP?$AAl?$AAa?$AAy?$AAb?$AAa?$AAc?$AAk?$AA?$AA@ 100015dc     esai_common_topaz_v1:mixerdrv.obj
 0001:000005f0       ??_C@_1BA@EEOGCIBB@?$AAL?$AAi?$AAn?$AAe?$AA?5?$AAI?$AAn?$AA?$AA@ 100015f0     esai_common_topaz_v1:mixerdrv.obj
 0001:00000600       ??_C@_1BG@OGJPAHBK@?$AAM?$AAi?$AAc?$AAr?$AAo?$AAp?$AAh?$AAo?$AAn?$AAe?$AA?$AA@ 10001600     esai_common_topaz_v1:mixerdrv.obj
 0001:00000618       ??_C@_1CE@BJPEGCKG@?$AAR?$AAe?$AAc?$AAo?$AAr?$AAd?$AAi?$AAn?$AAg?$AA?5?$AAC?$AAo?$AAn?$AAt?$AAr?$AAo?$AAl?$AA?$AA@ 10001618     esai_common_topaz_v1:mixerdrv.obj
 0001:0000063c       ??_C@_1CA@KOFAABPH@?$AAR?$AAe?$AAc?$AAo?$AAr?$AAd?$AAi?$AAn?$AAg?$AA?5?$AAC?$AAo?$AAn?$AAt?$AAr?$AA?$AA@ 1000163c     esai_common_topaz_v1:mixerdrv.obj
 0001:0000065c       ??_C@_1CC@OALPFLIM@?$AAP?$AAl?$AAa?$AAy?$AAb?$AAa?$AAc?$AAk?$AA?5?$AAC?$AAo?$AAn?$AAt?$AAr?$AAo?$AAl?$AA?$AA@ 1000165c     esai_common_topaz_v1:mixerdrv.obj
 0001:00000680       ??_C@_1BO@OJJBHHKI@?$AAP?$AAl?$AAa?$AAy?$AAb?$AAa?$AAc?$AAk?$AA?5?$AAC?$AAo?$AAn?$AAt?$AAr?$AA?$AA@ 10001680     esai_common_topaz_v1:mixerdrv.obj
 0001:0000075c       ??_7MixerControl@@6B@      1000175c     esai_common_topaz_v1:mixerdrv.obj
 0001:00000778       ??_7MixerControlVolumeMaster@@6B@ 10001778     esai_common_topaz_v1:mixerdrv.obj
 0001:0000079c       ??_C@_1BM@DBCMFCBE@?$AAM?$AAa?$AAs?$AAt?$AAe?$AAr?$AA?5?$AAV?$AAo?$AAl?$AAu?$AAm?$AAe?$AA?$AA@ 1000179c     esai_common_topaz_v1:mixerdrv.obj
 0001:000007b8       ??_7MixerControlVolumeMic@@6B@ 100017b8     esai_common_topaz_v1:mixerdrv.obj
 0001:000007dc       ??_C@_1BG@LAGONMFD@?$AAM?$AAi?$AAc?$AA?5?$AAV?$AAo?$AAl?$AAu?$AAm?$AAe?$AA?$AA@ 100017dc     esai_common_topaz_v1:mixerdrv.obj
 0001:000007f4       ??_7MixerControlMuteMaster@@6B@ 100017f4     esai_common_topaz_v1:mixerdrv.obj
 0001:00000818       ??_C@_1BI@PEAJCPFH@?$AAM?$AAa?$AAs?$AAt?$AAe?$AAr?$AA?5?$AAM?$AAu?$AAt?$AAe?$AA?$AA@ 10001818     esai_common_topaz_v1:mixerdrv.obj
 0001:00000830       ??_7MixerControlMuteMic@@6B@ 10001830     esai_common_topaz_v1:mixerdrv.obj
 0001:00000854       ??_C@_1BC@MOMKCGGI@?$AAM?$AAi?$AAc?$AA?5?$AAM?$AAu?$AAt?$AAe?$AA?$AA@ 10001854     esai_common_topaz_v1:mixerdrv.obj
 0001:00000868       ??_7MixerControlLoopback@@6B@ 10001868     esai_common_topaz_v1:mixerdrv.obj
 0001:0000088c       ??_C@_1CC@NMFCMAHN@?$AAL?$AAo?$AAo?$AAp?$AAb?$AAa?$AAc?$AAk?$AA?5?$AAC?$AAo?$AAn?$AAt?$AAr?$AAo?$AAl?$AA?$AA@ 1000188c     esai_common_topaz_v1:mixerdrv.obj
 0001:000008b0       ??_C@_1BC@NMCMBANA@?$AAL?$AAo?$AAo?$AAp?$AAb?$AAa?$AAc?$AAk?$AA?$AA@ 100018b0     esai_common_topaz_v1:mixerdrv.obj
 0001:000008c4       ??_7MixerControlInputMux@@6B@ 100018c4     esai_common_topaz_v1:mixerdrv.obj
 0001:000008e0       ??_7MixerControlList@@6B@  100018e0     esai_common_topaz_v1:mixerdrv.obj
 0001:000008e4       ??_C@_1BI@DKACBKCL@?$AAA?$AAu?$AAd?$AAi?$AAo?$AA?5?$AAM?$AAi?$AAx?$AAe?$AAr?$AA?$AA@ 100018e4     esai_common_topaz_v1:mixerdrv.obj
 0001:000008fc       ??_C@_1BE@FNMPOHBO@?$AAI?$AAn?$AAp?$AAu?$AAt?$AA?5?$AAM?$AAu?$AAx?$AA?$AA@ 100018fc     esai_common_topaz_v1:mixerdrv.obj
 0001:00000938       ??0CWM8580@@QAA@XZ         10001938 f   wm8580.obj
 0001:00000960       ??1CWM8580@@QAA@XZ         10001960 f   wm8580.obj
 0001:00000968       ?ReadRegister@CWM8580@@AAAEK@Z 10001968 f   wm8580.obj
 0001:00000a38       ?WriteRegister@CWM8580@@AAAHKK@Z 10001a38 f   wm8580.obj
 0001:00000b08       ?GetDeviceID@CWM8580@@QAAHXZ 10001b08 f   wm8580.obj
 0001:00000b48       ?ConfigOutput@CWM8580@@QAAHKKKKW4AUDIO_PROTOCOL@@@Z 10001b48 f   wm8580.obj
 0001:00000df0       ?EnableDAC@CWM8580@@QAAHXZ 10001df0 f   wm8580.obj
 0001:00000e48       ?DisableDAC@CWM8580@@QAAHXZ 10001e48 f   wm8580.obj
 0001:00000e8c       ?SetOutputGain@CWM8580@@QAAHKKKK@Z 10001e8c f   wm8580.obj
 0001:00000f2c       ?GetDACBitClock@CWM8580@@QAAIXZ 10001f2c f   wm8580.obj
 0001:00000fac       ?EnableCLKO@CWM8580@@QAAHXZ 10001fac f   wm8580.obj
 0001:0000107c       ?InitCodec@CWM8580@@QAAHXZ 1000207c f   wm8580.obj
 0001:00001100       ??0CAK5702@@QAA@XZ         10002100 f   ak5702.obj
 0001:00001140       ??1CAK5702@@QAA@XZ         10002140 f   ak5702.obj
 0001:00001148       ?WriteRegister@CAK5702@@AAAHEE@Z 10002148 f   ak5702.obj
 0001:000011bc       ?InitAK5702@CAK5702@@QAAHXZ 100021bc f   ak5702.obj
 0001:000012a0       ?DisableADC@CAK5702@@QAAHXZ 100022a0 f   ak5702.obj
 0001:00001324       ?SetPLLPower@CAK5702@@QAAXH@Z 10002324 f   ak5702.obj
 0001:00001388       ?SetCodecPower@CAK5702@@QAAXW4AK5702_POWER_MODE@@@Z 10002388 f   ak5702.obj
 0001:00001474       ?SetInputGain@CAK5702@@QAAXEEEEK@Z 10002474 f   ak5702.obj
 0001:000014e4       ?ConfigADC@CAK5702@@QAAHW4AUDIO_PROTOCOL@@KKKKW4AK5702_PLL_MODE@@@Z 100024e4 f   ak5702.obj
 0001:0000167c       ?EnalbeADC@CAK5702@@QAAHXZ 1000267c f   ak5702.obj
 0001:0000173c       ?BSPAudioInitCodec@@YAHXZ  1000273c f   bsphwctxt.obj
 0001:00001848       ?BSPAudioConfigDAC@@YAHKKKKW4AUDIO_PROTOCOL@@@Z 10002848 f   bsphwctxt.obj
 0001:00001888       ?BSPAudioConfigADC@@YAHKKKKW4AUDIO_PROTOCOL@@@Z 10002888 f   bsphwctxt.obj
 0001:000018d0       ?BSPAudioStartDAC@@YAXXZ   100028d0 f   bsphwctxt.obj
 0001:000018e0       ?BSPAudioStopDAC@@YAXXZ    100028e0 f   bsphwctxt.obj
 0001:000018f0       ?BSPAudioStartADC@@YAXXZ   100028f0 f   bsphwctxt.obj
 0001:00001900       ?BSPAudioStopADC@@YAXXZ    10002900 f   bsphwctxt.obj
 0001:00001910       ?BSPAudioSetOutputGain@@YAXK@Z 10002910 f   bsphwctxt.obj
 0001:00001944       ?BSPAudioSetInputGain@@YAXK@Z 10002944 f   bsphwctxt.obj
 0001:0000198c       ?BSPAudioGetInputDeviceNum@@YAEXZ 1000298c f   bsphwctxt.obj
 0001:00001994       ?BSPAllocOutputDMABuffer@@YAGPAPAEPAT_LARGE_INTEGER@@@Z 10002994 f   bsphwctxt.obj
 0001:000019e4       ?BSPDeallocOutputDMABuffer@@YAXPAET_LARGE_INTEGER@@@Z 100029e4 f   bsphwctxt.obj
 0001:00001a48       ?BSPAllocInputDMABuffer@@YAGPAPAEPAT_LARGE_INTEGER@@@Z 10002a48 f   bsphwctxt.obj
 0001:00001a98       ?BSPDeallocInputDMABuffer@@YAXPAET_LARGE_INTEGER@@@Z 10002a98 f   bsphwctxt.obj
 0001:00001afc       ?BSPAudioIomuxConfig@@YAXXZ 10002afc f   bsphwctxt.obj
 0001:00001bc4       ?BSPESAIEnableClock@@YAHIH@Z 10002bc4 f   bsphwctxt.obj
 0001:00001c14       ?BSPAudioGetSdmaPriority@@YAEXZ 10002c14 f   bsphwctxt.obj
 0001:00001c1c       ?BSPAudioPowerUp@@YAXH@Z   10002c1c f   bsphwctxt.obj
 0001:00001c20       ?BSPAudioPowerDown@@YAXH@Z 10002c20 f   bsphwctxt.obj
 0001:00001c24       ?BSPAudioGetOutputProtocol@@YA?AW4AUDIO_PROTOCOL@@XZ 10002c24 f   bsphwctxt.obj
 0001:00001c34       ?BSPAudioGetInputProtocol@@YA?AW4AUDIO_PROTOCOL@@XZ 10002c34 f   bsphwctxt.obj
 0001:00001c44       ?BSPIsSupportedOutputFormat@@YAHPAUWAVEFORMATEXTENSIBLE@@@Z 10002c44 f   bsphwctxt.obj
 0001:00001d98       ?BSPIsSupportedInputFormat@@YAHPAUWAVEFORMATEXTENSIBLE@@@Z 10002d98 f   bsphwctxt.obj
 0001:00001eec       ?BSPAudioGetTxBitClock@@YAIXZ 10002eec f   bsphwctxt.obj
 0001:00001efc       ?BSPAudioDeinitCodec@@YAXXZ 10002efc f   bsphwctxt.obj
 0001:00001f58       WAV_Init                   10002f58 f   esai_common_topaz_v1:wavemain.obj
 0001:00001f5c       WAV_Deinit                 10002f5c f   esai_common_topaz_v1:wavemain.obj
 0001:00001f6c       WAV_Open                   10002f6c f   esai_common_topaz_v1:wavemain.obj
 0001:00001f8c       WAV_Close                  10002f8c f   esai_common_topaz_v1:wavemain.obj
 0001:00001fa4       ?HandleWaveMessage@@YAHPAUMMDRV_MESSAGE_PARAMS@@PAK@Z 10002fa4 f   esai_common_topaz_v1:wavemain.obj
 0001:00002394       WAV_IOControl              10003394 f   esai_common_topaz_v1:wavemain.obj
 0001:000024a0       ?InitESAI@HardwareContext@@AAAXXZ 100034a0 f   esai_common_topaz_v1:hwctxt.obj
 0001:000024e4       ?ConfigESAITx@HardwareContext@@AAAXXZ 100034e4 f   esai_common_topaz_v1:hwctxt.obj
 0001:000025ec       ?ConfigESAIRx@HardwareContext@@AAAXXZ 100035ec f   esai_common_topaz_v1:hwctxt.obj
 0001:000026d0       ?InitOutputDMA@HardwareContext@@AAAHXZ 100036d0 f   esai_common_topaz_v1:hwctxt.obj
 0001:00002798       ?ConfigOutputDMA@HardwareContext@@AAAHXZ 10003798 f   esai_common_topaz_v1:hwctxt.obj
 0001:0000285c       ?InitInputDMA@HardwareContext@@AAAHXZ 1000385c f   esai_common_topaz_v1:hwctxt.obj
 0001:00002944       ?ConfigInputDMA@HardwareContext@@AAAHXZ 10003944 f   esai_common_topaz_v1:hwctxt.obj
 0001:00002a10       ?StopCodec@HardwareContext@@AAAXW4AUDIO_BUS@@@Z 10003a10 f   esai_common_topaz_v1:hwctxt.obj
 0001:00002acc       ?PrepareESAI@HardwareContext@@AAAXW4AUDIO_BUS@@@Z 10003acc f   esai_common_topaz_v1:hwctxt.obj
 0001:00002bb8       ?StartESAI@HardwareContext@@AAAXW4AUDIO_BUS@@@Z 10003bb8 f   esai_common_topaz_v1:hwctxt.obj
 0001:00002c98       ?StopESAI@HardwareContext@@AAAXW4AUDIO_BUS@@@Z 10003c98 f   esai_common_topaz_v1:hwctxt.obj
 0001:00002d44       ?StopOutputDMA@HardwareContext@@QAAXXZ 10003d44 f   esai_common_topaz_v1:hwctxt.obj
 0001:00002dc4       ?StartInputDMA@HardwareContext@@QAAHXZ 10003dc4 f   esai_common_topaz_v1:hwctxt.obj
 0001:00002e6c       ?StopInputDMA@HardwareContext@@QAAXXZ 10003e6c f   esai_common_topaz_v1:hwctxt.obj
 0001:00002ec4       ?TransferBuffer@HardwareContext@@IAAKW4AUDIO_BUS@@E@Z 10003ec4 f   esai_common_topaz_v1:hwctxt.obj
 0001:00002f54       ?DisableDelayThread@HardwareContext@@QAAXXZ 10003f54 f   esai_common_topaz_v1:hwctxt.obj
 0001:00003054       ?CallDisableDelayThread@@YAXPAVHardwareContext@@@Z 10004054 f   esai_common_topaz_v1:hwctxt.obj
 0001:00003058       ?SetOutputGain@HardwareContext@@QAAIK@Z 10004058 f   esai_common_topaz_v1:hwctxt.obj
 0001:0000307c       ?SetOutputMute@HardwareContext@@QAAIH@Z 1000407c f   esai_common_topaz_v1:hwctxt.obj
 0001:0000309c       ?GetOutputGain@HardwareContext@@QAAKXZ 1000409c f   esai_common_topaz_v1:hwctxt.obj
 0001:000030a4       ?GetOutputMute@HardwareContext@@QAAHXZ 100040a4 f   esai_common_topaz_v1:hwctxt.obj
 0001:000030ac       ?GetInputMute@HardwareContext@@QAAHXZ 100040ac f   esai_common_topaz_v1:hwctxt.obj
 0001:000030b4       ?SetInputMute@HardwareContext@@QAAIH@Z 100040b4 f   esai_common_topaz_v1:hwctxt.obj
 0001:000030d4       ?GetInputGain@HardwareContext@@QAAKXZ 100040d4 f   esai_common_topaz_v1:hwctxt.obj
 0001:000030dc       ?SetInputGain@HardwareContext@@QAAIK@Z 100040dc f   esai_common_topaz_v1:hwctxt.obj
 0001:00003100       ?PowerDown@HardwareContext@@QAAXXZ 10004100 f   esai_common_topaz_v1:hwctxt.obj
 0001:0000316c       ?GetDriverRegValue@HardwareContext@@QAAKPAGK@Z 1000416c f   esai_common_topaz_v1:hwctxt.obj
 0001:000031d0       ?IsSupportedOutputFormat@HardwareContext@@QAAHPAUtWAVEFORMATEX@@@Z 100041d0 f   esai_common_topaz_v1:hwctxt.obj
 0001:00003258       ?IsSupportedInputFormat@HardwareContext@@QAAHPAUtWAVEFORMATEX@@@Z 10004258 f   esai_common_topaz_v1:hwctxt.obj
 0001:000032a4       ?InitInputWaveFormat@HardwareContext@@QAAHPAUtWAVEFORMATEX@@@Z 100042a4 f   esai_common_topaz_v1:hwctxt.obj
 0001:00003360       ?DeinitInputWaveFormat@HardwareContext@@QAAHPAUtWAVEFORMATEX@@@Z 10004360 f   esai_common_topaz_v1:hwctxt.obj
 0001:00003370       ?DeinitOutputWaveFormat@HardwareContext@@QAAHPAUtWAVEFORMATEX@@@Z 10004370 f   esai_common_topaz_v1:hwctxt.obj
 0001:00003380       ?ForceSpeaker@HardwareContext@@QAAKH@Z 10004380 f   esai_common_topaz_v1:hwctxt.obj
 0001:00003388       ?SelectInputSource@HardwareContext@@QAAHK@Z 10004388 f   esai_common_topaz_v1:hwctxt.obj
 0001:00003390       ?DeinitAsrcP2P@HardwareContext@@AAAXXZ 10004390 f   esai_common_topaz_v1:hwctxt.obj
 0001:000033e4       ?ConfigAsrc@HardwareContext@@AAAHXZ 100043e4 f   esai_common_topaz_v1:hwctxt.obj
 0001:00003554       ??0HardwareContext@@QAA@XZ 10004554 f   esai_common_topaz_v1:hwctxt.obj
 0001:000035a4       ?Deinit@HardwareContext@@QAAHXZ 100045a4 f   esai_common_topaz_v1:hwctxt.obj
 0001:00003628       ?InitDisableDelayThread@HardwareContext@@IAAHXZ 10004628 f   esai_common_topaz_v1:hwctxt.obj
 0001:00003728       ?TransferOutputBuffers@HardwareContext@@IAAKXZ 10004728 f   esai_common_topaz_v1:hwctxt.obj
 0001:00003794       ?TransferInputBuffers@HardwareContext@@IAAKE@Z 10004794 f   esai_common_topaz_v1:hwctxt.obj
 0001:0000389c       ?OutputIntrRoutine@HardwareContext@@AAAXXZ 1000489c f   esai_common_topaz_v1:hwctxt.obj
 0001:000039b0       ?InputIntrRoutine@HardwareContext@@AAAXXZ 100049b0 f   esai_common_topaz_v1:hwctxt.obj
 0001:00003b34       ?InitOutputWaveFormat@HardwareContext@@QAAHPAUtWAVEFORMATEX@@@Z 10004b34 f   esai_common_topaz_v1:hwctxt.obj
 0001:00003cc0       ?AsrcIntrRoutine@HardwareContext@@AAAXXZ 10004cc0 f   esai_common_topaz_v1:hwctxt.obj
 0001:00003de0       ?StartOutputDMA@HardwareContext@@QAAHXZ 10004de0 f   esai_common_topaz_v1:hwctxt.obj
 0001:00003f3c       ?InterruptThread@HardwareContext@@QAAXXZ 10004f3c f   esai_common_topaz_v1:hwctxt.obj
 0001:00003fbc       ?CallInterruptThread@@YAXPAVHardwareContext@@@Z 10004fbc f   esai_common_topaz_v1:hwctxt.obj
 0001:00003fc0       ?PowerUp@HardwareContext@@QAAXXZ 10004fc0 f   esai_common_topaz_v1:hwctxt.obj
 0001:00004004       ?AsrcIntrThread@HardwareContext@@QAAXXZ 10005004 f   esai_common_topaz_v1:hwctxt.obj
 0001:000040c0       ?InitInterruptThread@HardwareContext@@IAAHXZ 100050c0 f   esai_common_topaz_v1:hwctxt.obj
 0001:0000416c       ?PmControlMessage@HardwareContext@@QAAHKPAEK0KPAK@Z 1000516c f   esai_common_topaz_v1:hwctxt.obj
 0001:000042a4       ?CallAsrcIntrThread@@YAXPAVHardwareContext@@@Z 100052a4 f   esai_common_topaz_v1:hwctxt.obj
 0001:000042a8       ?InitAsrcP2P@HardwareContext@@AAAHXZ 100052a8 f   esai_common_topaz_v1:hwctxt.obj
 0001:00004494       ?Init@HardwareContext@@QAAHK@Z 10005494 f   esai_common_topaz_v1:hwctxt.obj
 0001:000045cc       ?CreateHWContext@HardwareContext@@SAHK@Z 100055cc f   esai_common_topaz_v1:hwctxt.obj
 0001:00004624       ??0DeviceContext@@QAA@XZ   10005624 f   esai_common_topaz_v1:devctxt.obj
 0001:0000466c       ?GetGain@DeviceContext@@QAAKXZ 1000566c f   esai_common_topaz_v1:devctxt.obj
 0001:00004674       ?GetDefaultStreamGain@DeviceContext@@QAAKXZ 10005674 f   esai_common_topaz_v1:devctxt.obj
 0001:0000467c       ?GetSecondaryGainLimit@DeviceContext@@QAAKK@Z 1000567c f   esai_common_topaz_v1:devctxt.obj
 0001:00004688       ?IsSupportedFormat@DeviceContext@@UAAHPAUtWAVEFORMATEX@@@Z 10005688 f   esai_common_topaz_v1:devctxt.obj
 0001:0000471c       ?IsSupportedFormat@OutputDeviceContext@@UAAHPAUtWAVEFORMATEX@@@Z 1000571c f   esai_common_topaz_v1:devctxt.obj
 0001:00004770       ?IsSupportedFormat@InputDeviceContext@@UAAHPAUtWAVEFORMATEX@@@Z 10005770 f   esai_common_topaz_v1:devctxt.obj
 0001:00004794       ?DeinitDeviceWaveFormat@DeviceContext@@UAAHPAUtWAVEFORMATEX@@@Z 10005794 f   esai_common_topaz_v1:devctxt.obj
 0001:0000479c       ?DeinitDeviceWaveFormat@OutputDeviceContext@@UAAHPAUtWAVEFORMATEX@@@Z 1000579c f   esai_common_topaz_v1:devctxt.obj
 0001:000047ac       ?DeinitDeviceWaveFormat@InputDeviceContext@@UAAHPAUtWAVEFORMATEX@@@Z 100057ac f   esai_common_topaz_v1:devctxt.obj
 0001:000047bc       ?InitDeviceWaveFormat@DeviceContext@@UAAHPAUtWAVEFORMATEX@@@Z 100057bc f   esai_common_topaz_v1:devctxt.obj
 0001:000047c4       ?InitDeviceWaveFormat@OutputDeviceContext@@UAAHPAUtWAVEFORMATEX@@@Z 100057c4 f   esai_common_topaz_v1:devctxt.obj
 0001:000047d4       ?InitDeviceWaveFormat@InputDeviceContext@@UAAHPAUtWAVEFORMATEX@@@Z 100057d4 f   esai_common_topaz_v1:devctxt.obj
 0001:000047e4       ?NewStream@DeviceContext@@UAAKPAVStreamContext@@@Z 100057e4 f   esai_common_topaz_v1:devctxt.obj
 0001:00004858       ?DeleteStream@DeviceContext@@QAAXPAVStreamContext@@@Z 10005858 f   esai_common_topaz_v1:devctxt.obj
 0001:000048bc       ?TransferBuffer@DeviceContext@@QAAPAEPAE0PAUTRANSFER_STATUS@@@Z 100058bc f   esai_common_topaz_v1:devctxt.obj
 0001:00004954       ?RecalcAllGains@DeviceContext@@QAAXXZ 10005954 f   esai_common_topaz_v1:devctxt.obj
 0001:00004984       ?StreamReadyToRender@OutputDeviceContext@@UAAXPAVStreamContext@@@Z 10005984 f   esai_common_topaz_v1:devctxt.obj
 0001:00004994       ?StreamReadyToRender@InputDeviceContext@@UAAXPAVStreamContext@@@Z 10005994 f   esai_common_topaz_v1:devctxt.obj
 0001:000049a4       ?GetDevCaps@OutputDeviceContext@@UAAKPAXK@Z 100059a4 f   esai_common_topaz_v1:devctxt.obj
 0001:000049c8       ?GetDevCaps@InputDeviceContext@@UAAKPAXK@Z 100059c8 f   esai_common_topaz_v1:devctxt.obj
 0001:000049ec       ?GetExtDevCaps@OutputDeviceContext@@UAAKPAXK@Z 100059ec f   esai_common_topaz_v1:devctxt.obj
 0001:00004a10       ?GetExtDevCaps@InputDeviceContext@@UAAKPAXK@Z 10005a10 f   esai_common_topaz_v1:devctxt.obj
 0001:00004a18       ?OpenStream@DeviceContext@@QAAKPAUwaveopendesc_tag@@KPAPAVStreamContext@@@Z 10005a18 f   esai_common_topaz_v1:devctxt.obj
 0001:00004b20       ?ResetBaseInfo@DeviceContext@@QAAXXZ 10005b20 f   esai_common_topaz_v1:devctxt.obj
 0001:00004b50       ?GetBaseSampleRate@DeviceContext@@QAAKXZ 10005b50 f   esai_common_topaz_v1:devctxt.obj
 0001:00004b58       ?GetBaseSampleRateInverse@DeviceContext@@QAAKXZ 10005b58 f   esai_common_topaz_v1:devctxt.obj
 0001:00004b60       ?GetChannels@OutputDeviceContext@@UAAKXZ 10005b60 f   esai_common_topaz_v1:devctxt.obj
 0001:00004b68       ?GetChannels@InputDeviceContext@@UAAKXZ 10005b68 f   esai_common_topaz_v1:devctxt.obj
 0001:00004b70       ?GetNativeFormat@DeviceContext@@QAAKKPAXKPAK@Z 10005b70 f   esai_common_topaz_v1:devctxt.obj
 0001:00004c24       ?GetProperty@DeviceContext@@QAAKPAUtag_WAVEPROPINFO@@@Z 10005c24 f   esai_common_topaz_v1:devctxt.obj
 0001:00004d08       ?SetProperty@DeviceContext@@QAAKPAUtag_WAVEPROPINFO@@@Z 10005d08 f   esai_common_topaz_v1:devctxt.obj
 0001:00004d10       ?SetSecondaryGainLimit@DeviceContext@@QAAKKK@Z 10005d10 f   esai_common_topaz_v1:devctxt.obj
 0001:00004d34       ??_GOutputStreamContextEx@@UAAPAXI@Z 10005d34 f i esai_common_topaz_v1:devctxt.obj
 0001:00004d34       ??_EOutputStreamContextEx@@UAAPAXI@Z 10005d34 f i esai_common_topaz_v1:devctxt.obj
 0001:00004d58       ??_EOutputStreamContextM8@@UAAPAXI@Z 10005d58 f i esai_common_topaz_v1:devctxt.obj
 0001:00004d58       ??_GOutputStreamContextM8@@UAAPAXI@Z 10005d58 f i esai_common_topaz_v1:devctxt.obj
 0001:00004d7c       ??_EOutputStreamContextS8@@UAAPAXI@Z 10005d7c f i esai_common_topaz_v1:devctxt.obj
 0001:00004d7c       ??_GOutputStreamContextS8@@UAAPAXI@Z 10005d7c f i esai_common_topaz_v1:devctxt.obj
 0001:00004da0       ??_GOutputStreamContextM16@@UAAPAXI@Z 10005da0 f i esai_common_topaz_v1:devctxt.obj
 0001:00004da0       ??_EOutputStreamContextM16@@UAAPAXI@Z 10005da0 f i esai_common_topaz_v1:devctxt.obj
 0001:00004dc4       ??_EOutputStreamContextS16@@UAAPAXI@Z 10005dc4 f i esai_common_topaz_v1:devctxt.obj
 0001:00004dc4       ??_GOutputStreamContextS16@@UAAPAXI@Z 10005dc4 f i esai_common_topaz_v1:devctxt.obj
 0001:00004de8       ?SetBaseSampleRate@DeviceContext@@UAAXK@Z 10005de8 f   esai_common_topaz_v1:devctxt.obj
 0001:00004e20       ??_EInputStreamContextEx@@UAAPAXI@Z 10005e20 f i esai_common_topaz_v1:devctxt.obj
 0001:00004e20       ??_GInputStreamContextEx@@UAAPAXI@Z 10005e20 f i esai_common_topaz_v1:devctxt.obj
 0001:00004e44       ?CreateStream@OutputDeviceContext@@UAAPAVStreamContext@@PAUwaveopendesc_tag@@@Z 10005e44 f   esai_common_topaz_v1:devctxt.obj
 0001:00004fbc       ?CreateStream@InputDeviceContext@@UAAPAVStreamContext@@PAUwaveopendesc_tag@@@Z 10005fbc f   esai_common_topaz_v1:devctxt.obj
 0001:0000502c       ??0StreamContext@@QAA@XZ   1000602c f   esai_common_topaz_v1:strmctxt.obj
 0001:00005040       ??1StreamContext@@UAA@XZ   10006040 f   esai_common_topaz_v1:strmctxt.obj
 0001:00005050       ?GetDeviceContext@StreamContext@@QAAPAVDeviceContext@@XZ 10006050 f   esai_common_topaz_v1:strmctxt.obj
 0001:00005058       ?DoDriverCallback@StreamContext@@QAAXIKK@Z 10006058 f   esai_common_topaz_v1:strmctxt.obj
 0001:00005088       ?DoCallbackReturnBuffer@StreamContext@@UAAXPAUwavehdr_tag@@@Z 10006088 f   esai_common_topaz_v1:strmctxt.obj
 0001:000050c0       ?DoCallbackStreamOpened@StreamContext@@UAAXXZ 100060c0 f   esai_common_topaz_v1:strmctxt.obj
 0001:000050f8       ?DoCallbackStreamClosed@StreamContext@@UAAXXZ 100060f8 f   esai_common_topaz_v1:strmctxt.obj
 0001:0000512c       ?SetSecondaryGainClass@StreamContext@@QAAKK@Z 1000612c f   esai_common_topaz_v1:strmctxt.obj
 0001:0000515c       ?IsExclusive@StreamContext@@UAAHXZ 1000615c f   esai_common_topaz_v1:strmctxt.obj
 0001:00005164       ?Open@StreamContext@@UAAKPAVDeviceContext@@PAUwaveopendesc_tag@@K@Z 10006164 f   esai_common_topaz_v1:strmctxt.obj
 0001:0000529c       ?AddRef@StreamContext@@QAAJXZ 1000629c f   esai_common_topaz_v1:strmctxt.obj
 0001:000052b0       ?Release@StreamContext@@QAAJXZ 100062b0 f   esai_common_topaz_v1:strmctxt.obj
 0001:000052f4       ?QueueBuffer@StreamContext@@UAAKPAUwavehdr_tag@@@Z 100062f4 f   esai_common_topaz_v1:strmctxt.obj
 0001:00005398       ?GetNextBuffer@StreamContext@@QAAPAEXZ 10006398 f   esai_common_topaz_v1:strmctxt.obj
 0001:00005468       ?BreakLoop@StreamContext@@QAAKXZ 10006468 f   esai_common_topaz_v1:strmctxt.obj
 0001:000054f4       ?MapGain@StreamContext@@QAAKKK@Z 100064f4 f   esai_common_topaz_v1:strmctxt.obj
 0001:000055b0       ?GetPos@StreamContext@@UAAKPAUmmtime_tag@@@Z 100065b0 f   esai_common_topaz_v1:strmctxt.obj
 0001:00005690       ?Open@WaveStreamContext@@UAAKPAVDeviceContext@@PAUwaveopendesc_tag@@K@Z 10006690 f   esai_common_topaz_v1:strmctxt.obj
 0001:00005774       ?GetRate@WaveStreamContext@@QAAKPAK@Z 10006774 f   esai_common_topaz_v1:strmctxt.obj
 0001:00005784       ?Run@StreamContext@@UAAKXZ 10006784 f   esai_common_topaz_v1:strmctxt.obj
 0001:000057b4       ?Stop@StreamContext@@UAAKXZ 100067b4 f   esai_common_topaz_v1:strmctxt.obj
 0001:000057c4       ?Reset@StreamContext@@UAAKXZ 100067c4 f   esai_common_topaz_v1:strmctxt.obj
 0001:00005854       ?SetRate@WaveStreamContext@@UAAKK@Z 10006854 f   esai_common_topaz_v1:strmctxt.obj
 0001:000058b8       ?Render@WaveStreamContext@@UAAPAEPAE00PAUTRANSFER_STATUS@@@Z 100068b8 f   esai_common_topaz_v1:strmctxt.obj
 0001:000059b4       ?ClearBuffer@StreamContext@@SAXPAE0@Z 100069b4 f   esai_common_topaz_v1:strmctxt.obj
 0001:000059c0       ?GetProperty@StreamContext@@QAAKPAUtag_WAVEPROPINFO@@@Z 100069c0 f   esai_common_topaz_v1:strmctxt.obj
 0001:000059c8       ?SetProperty@StreamContext@@QAAKPAUtag_WAVEPROPINFO@@@Z 100069c8 f   esai_common_topaz_v1:strmctxt.obj
 0001:000059d0       ??_EStreamContext@@UAAPAXI@Z 100069d0 f i esai_common_topaz_v1:strmctxt.obj
 0001:000059d0       ??_GStreamContext@@UAAPAXI@Z 100069d0 f i esai_common_topaz_v1:strmctxt.obj
 0001:000059f4       ?GainChange@StreamContext@@UAAXXZ 100069f4 f   esai_common_topaz_v1:strmctxt.obj
 0001:00005a2c       ?Close@StreamContext@@UAAKXZ 10006a2c f   esai_common_topaz_v1:strmctxt.obj
 0001:00005a80       ?LookupMxLine@@YAPBUtagMXLINEDESC@@G@Z 10006a80 f   esai_common_topaz_v1:mixerdrv.obj
 0001:00005ac4       ?SetControlID@MixerControl@@UAAXK@Z 10006ac4 f i esai_common_topaz_v1:mixerdrv.obj
 0001:00005acc       ?CopyMixerControl@MixerControl@@UAAXPAUtMIXERCONTROL@@@Z 10006acc f i esai_common_topaz_v1:mixerdrv.obj
 0001:00005b3c       ?GetControlDetails@MixerControl@@UAAKPAUtMIXERCONTROLDETAILS@@K@Z 10006b3c f i esai_common_topaz_v1:mixerdrv.obj
 0001:00005b44       ?SetControlDetails@MixerControl@@UAAKPAUtMIXERCONTROLDETAILS@@K@Z 10006b44 f i esai_common_topaz_v1:mixerdrv.obj
 0001:00005b4c       ??_EMixerControl@@UAAPAXI@Z 10006b4c f i esai_common_topaz_v1:mixerdrv.obj
 0001:00005b4c       ??_GMixerControl@@UAAPAXI@Z 10006b4c f i esai_common_topaz_v1:mixerdrv.obj
 0001:00005b70       ?CopyMixerControl@MixerControlVolume@@UAAXPAUtMIXERCONTROL@@@Z 10006b70 f i esai_common_topaz_v1:mixerdrv.obj
 0001:00005bdc       ?GetControlType@MixerControlVolume@@UAAKXZ 10006bdc f i esai_common_topaz_v1:mixerdrv.obj
 0001:00005be8       ?GetControlDetails@MixerControlVolume@@UAAKPAUtMIXERCONTROLDETAILS@@K@Z 10006be8 f i esai_common_topaz_v1:mixerdrv.obj
 0001:00005cd4       ?SetControlDetails@MixerControlVolume@@UAAKPAUtMIXERCONTROLDETAILS@@K@Z 10006cd4 f i esai_common_topaz_v1:mixerdrv.obj
 0001:00005dbc       ?CopyMixerControl@MixerControlVolumeMaster@@UAAXPAUtMIXERCONTROL@@@Z 10006dbc f i esai_common_topaz_v1:mixerdrv.obj
 0001:00005de8       ?GetLineID@MixerControlVolumeMaster@@UAAGXZ 10006de8 f i esai_common_topaz_v1:mixerdrv.obj
 0001:00005df4       ?SetGain@MixerControlVolumeMaster@@UAAXK@Z 10006df4 f i esai_common_topaz_v1:mixerdrv.obj
 0001:00005e04       ?GetGain@MixerControlVolumeMaster@@UAAKXZ 10006e04 f i esai_common_topaz_v1:mixerdrv.obj
 0001:00005e14       ?CopyMixerControl@MixerControlVolumeMic@@UAAXPAUtMIXERCONTROL@@@Z 10006e14 f i esai_common_topaz_v1:mixerdrv.obj
 0001:00005e40       ?GetLineID@MixerControlVolumeMic@@UAAGXZ 10006e40 f i esai_common_topaz_v1:mixerdrv.obj
 0001:00005e4c       ?SetGain@MixerControlVolumeMic@@UAAXK@Z 10006e4c f i esai_common_topaz_v1:mixerdrv.obj
 0001:00005e5c       ?GetGain@MixerControlVolumeMic@@UAAKXZ 10006e5c f i esai_common_topaz_v1:mixerdrv.obj
 0001:00005e6c       ?CopyMixerControl@MixerControlBoolean@@UAAXPAUtMIXERCONTROL@@@Z 10006e6c f i esai_common_topaz_v1:mixerdrv.obj
 0001:00005ed4       ?GetControlType@MixerControlBoolean@@UAAKXZ 10006ed4 f i esai_common_topaz_v1:mixerdrv.obj
 0001:00005ee0       ?GetControlDetails@MixerControlBoolean@@UAAKPAUtMIXERCONTROLDETAILS@@K@Z 10006ee0 f i esai_common_topaz_v1:mixerdrv.obj
 0001:00005f34       ?SetControlDetails@MixerControlBoolean@@UAAKPAUtMIXERCONTROLDETAILS@@K@Z 10006f34 f i esai_common_topaz_v1:mixerdrv.obj
 0001:00005f84       ?CopyMixerControl@MixerControlMuteMaster@@UAAXPAUtMIXERCONTROL@@@Z 10006f84 f i esai_common_topaz_v1:mixerdrv.obj
 0001:00005fb0       ?GetControlType@MixerControlMuteMaster@@UAAKXZ 10006fb0 f i esai_common_topaz_v1:mixerdrv.obj
 0001:00005fbc       ?GetLineID@MixerControlMuteMaster@@UAAGXZ 10006fbc f i esai_common_topaz_v1:mixerdrv.obj
 0001:00005fc8       ?GetValue@MixerControlMuteMaster@@UAAHXZ 10006fc8 f i esai_common_topaz_v1:mixerdrv.obj
 0001:00005fd8       ?SetValue@MixerControlMuteMaster@@UAAXH@Z 10006fd8 f i esai_common_topaz_v1:mixerdrv.obj
 0001:00005fe8       ?CopyMixerControl@MixerControlMuteMic@@UAAXPAUtMIXERCONTROL@@@Z 10006fe8 f i esai_common_topaz_v1:mixerdrv.obj
 0001:00006014       ?GetLineID@MixerControlMuteMic@@UAAGXZ 10007014 f i esai_common_topaz_v1:mixerdrv.obj
 0001:00006020       ?GetValue@MixerControlMuteMic@@UAAHXZ 10007020 f i esai_common_topaz_v1:mixerdrv.obj
 0001:00006030       ?SetValue@MixerControlMuteMic@@UAAXH@Z 10007030 f i esai_common_topaz_v1:mixerdrv.obj
 0001:00006040       ?CopyMixerControl@MixerControlLoopback@@UAAXPAUtMIXERCONTROL@@@Z 10007040 f i esai_common_topaz_v1:mixerdrv.obj
 0001:00006070       ?GetControlType@MixerControlLoopback@@UAAKXZ 10007070 f i esai_common_topaz_v1:mixerdrv.obj
 0001:0000607c       ?GetLineID@MixerControlLoopback@@UAAGXZ 1000707c f i esai_common_topaz_v1:mixerdrv.obj
 0001:00006088       ?GetValue@MixerControlLoopback@@UAAHXZ 10007088 f i esai_common_topaz_v1:mixerdrv.obj
 0001:00006090       ?SetValue@MixerControlLoopback@@UAAXH@Z 10007090 f i esai_common_topaz_v1:mixerdrv.obj
 0001:00006094       ?GetLineID@MixerControlInputMux@@UAAGXZ 10007094 f i esai_common_topaz_v1:mixerdrv.obj
 0001:000060a0       ?GetControlType@MixerControlInputMux@@UAAKXZ 100070a0 f i esai_common_topaz_v1:mixerdrv.obj
 0001:000060ac       ?GetListText@MixerControlInputMux@@QAAXPAUtMIXERCONTROLDETAILS_LISTTEXT@@K@Z 100070ac f i esai_common_topaz_v1:mixerdrv.obj
 0001:00006144       ?GetControlDetails@MixerControlInputMux@@UAAKPAUtMIXERCONTROLDETAILS@@K@Z 10007144 f i esai_common_topaz_v1:mixerdrv.obj
 0001:00006278       ?SetControlDetails@MixerControlInputMux@@UAAKPAUtMIXERCONTROLDETAILS@@K@Z 10007278 f i esai_common_topaz_v1:mixerdrv.obj
 0001:0000635c       ??0MixerControlList@@QAA@XZ 1000735c f i esai_common_topaz_v1:mixerdrv.obj
 0001:0000642c       ??_GMixerControlList@@UAAPAXI@Z 1000742c f i esai_common_topaz_v1:mixerdrv.obj
 0001:0000642c       ??_EMixerControlList@@UAAPAXI@Z 1000742c f i esai_common_topaz_v1:mixerdrv.obj
 0001:00006470       ?PerformMixerCallbacks@@YAXKK@Z 10007470 f   esai_common_topaz_v1:mixerdrv.obj
 0001:000064cc       ?wdev_MXDM_GETDEVCAPS@@YAKPAUtagMIXERCAPS@@K@Z 100074cc f   esai_common_topaz_v1:mixerdrv.obj
 0001:0000653c       ?wdev_MXDM_OPEN@@YAKPAKPAUtMIXEROPENDESC@@K@Z 1000753c f   esai_common_topaz_v1:mixerdrv.obj
 0001:000065cc       ?wdev_MXDM_CLOSE@@YAKK@Z   100075cc f   esai_common_topaz_v1:mixerdrv.obj
 0001:00006624       ?wdev_MXDM_GETLINEINFO@@YAKPAUtMIXERLINE@@K@Z 10007624 f   esai_common_topaz_v1:mixerdrv.obj
 0001:000069a8       ?wdev_MXDM_GETLINECONTROLS@@YAKPAUtMIXERLINECONTROLS@@K@Z 100079a8 f   esai_common_topaz_v1:mixerdrv.obj
 0001:00006c24       ?wdev_MXDM_GETCONTROLDETAILS@@YAKPAUtMIXERCONTROLDETAILS@@K@Z 10007c24 f   esai_common_topaz_v1:mixerdrv.obj
 0001:00006c90       ?wdev_MXDM_SETCONTROLDETAILS@@YAKPAUtMIXERCONTROLDETAILS@@K@Z 10007c90 f   esai_common_topaz_v1:mixerdrv.obj
 0001:00006d28       ?InitMixerControls@@YAHXZ  10007d28 f   esai_common_topaz_v1:mixerdrv.obj
 0001:00006d70       ?HandleMixerMessage@@YAHPAUMMDRV_MESSAGE_PARAMS@@PAK@Z 10007d70 f   esai_common_topaz_v1:mixerdrv.obj
 0001:00006e74       ??_GMixerControlVolumeMaster@@UAAPAXI@Z 10007e74 f i esai_common_topaz_v1:mixerdrv.obj
 0001:00006e74       ??_EMixerControlVolumeMaster@@UAAPAXI@Z 10007e74 f i esai_common_topaz_v1:mixerdrv.obj
 0001:00006e98       ??_EMixerControlVolumeMic@@UAAPAXI@Z 10007e98 f i esai_common_topaz_v1:mixerdrv.obj
 0001:00006e98       ??_GMixerControlVolumeMic@@UAAPAXI@Z 10007e98 f i esai_common_topaz_v1:mixerdrv.obj
 0001:00006ebc       ??_GMixerControlMuteMaster@@UAAPAXI@Z 10007ebc f i esai_common_topaz_v1:mixerdrv.obj
 0001:00006ebc       ??_EMixerControlMuteMaster@@UAAPAXI@Z 10007ebc f i esai_common_topaz_v1:mixerdrv.obj
 0001:00006ee0       ??_EMixerControlMuteMic@@UAAPAXI@Z 10007ee0 f i esai_common_topaz_v1:mixerdrv.obj
 0001:00006ee0       ??_GMixerControlMuteMic@@UAAPAXI@Z 10007ee0 f i esai_common_topaz_v1:mixerdrv.obj
 0001:00006f04       ??_GMixerControlLoopback@@UAAPAXI@Z 10007f04 f i esai_common_topaz_v1:mixerdrv.obj
 0001:00006f04       ??_EMixerControlLoopback@@UAAPAXI@Z 10007f04 f i esai_common_topaz_v1:mixerdrv.obj
 0001:00006f28       ?CopyMixerControl@MixerControlInputMux@@UAAXPAUtMIXERCONTROL@@@Z 10007f28 f i esai_common_topaz_v1:mixerdrv.obj
 0001:00006fb4       ??_GMixerControlInputMux@@UAAPAXI@Z 10007fb4 f i esai_common_topaz_v1:mixerdrv.obj
 0001:00006fb4       ??_EMixerControlInputMux@@UAAPAXI@Z 10007fb4 f i esai_common_topaz_v1:mixerdrv.obj
 0001:00006fd8       ?Open@OutputStreamContext@@UAAKPAVDeviceContext@@PAUwaveopendesc_tag@@K@Z 10007fd8 f   esai_common_topaz_v1:output.obj
 0001:00007014       ?Reset@OutputStreamContext@@UAAKXZ 10008014 f   esai_common_topaz_v1:output.obj
 0001:0000703c       ?ResetBaseInfo@OutputStreamContext@@UAAXXZ 1000803c f   esai_common_topaz_v1:output.obj
 0001:00007040       ?Render2@OutputStreamContextM8@@UAAPAEPAE00PAUTRANSFER_STATUS@@@Z 10008040 f   esai_common_topaz_v1:output.obj
 0001:000071c8       ?Render2@OutputStreamContextM16@@UAAPAEPAE00PAUTRANSFER_STATUS@@@Z 100081c8 f   esai_common_topaz_v1:output.obj
 0001:0000734c       ?Render2@OutputStreamContextS8@@UAAPAEPAE00PAUTRANSFER_STATUS@@@Z 1000834c f   esai_common_topaz_v1:output.obj
 0001:0000752c       ?Render2@OutputStreamContextS16@@UAAPAEPAE00PAUTRANSFER_STATUS@@@Z 1000852c f   esai_common_topaz_v1:output.obj
 0001:000076ec       ?Render2@OutputStreamContextEx@@UAAPAEPAE00PAUTRANSFER_STATUS@@@Z 100086ec f   esai_common_topaz_v1:output.obj
 0001:0000773c       ?Open@InputStreamContext@@UAAKPAVDeviceContext@@PAUwaveopendesc_tag@@K@Z 1000873c f   esai_common_topaz_v1:input.obj
 0001:00007758       ?DoCallbackReturnBuffer@InputStreamContext@@UAAXPAUwavehdr_tag@@@Z 10008758 f   esai_common_topaz_v1:input.obj
 0001:00007768       ?DoCallbackStreamOpened@InputStreamContext@@UAAXXZ 10008768 f   esai_common_topaz_v1:input.obj
 0001:0000777c       ?DoCallbackStreamClosed@InputStreamContext@@UAAXXZ 1000877c f   esai_common_topaz_v1:input.obj
 0001:00007790       ?Stop@InputStreamContext@@UAAKXZ 10008790 f   esai_common_topaz_v1:input.obj
 0001:000077c0       ?ResetBaseInfo@InputStreamContext@@UAAXXZ 100087c0 f   esai_common_topaz_v1:input.obj
 0001:000077c4       ?Render2@InputStreamContextEx@@UAAPAEPAE00PAUTRANSFER_STATUS@@@Z 100087c4 f   esai_common_topaz_v1:input.obj
 0001:00007814       ?GetESAIBaseRegAddr@@YAII@Z 10008814 f   esai_mx25_topaz_v1:mx25esai.obj
 0001:00007820       ?GetSdmaChannelIRQ@@YAKI@Z 10008820 f   esai_mx25_topaz_v1:mx25esai.obj
 0001:00007828       AsrcInit                   10008828 f   asrcbase_mx25_topaz_v1_stub:mx25asrc_stub.obj
 0001:00007830       AsrcDeinit                 10008830 f   asrcbase_mx25_topaz_v1_stub:mx25asrc_stub.obj
 0001:00007838       AsrcOpenPair               10008838 f   asrcbase_mx25_topaz_v1_stub:mx25asrc_stub.obj
 0001:00007840       AsrcStartConv              10008840 f   asrcbase_mx25_topaz_v1_stub:mx25asrc_stub.obj
 0001:00007848       AsrcStopConv               10008848 f   asrcbase_mx25_topaz_v1_stub:mx25asrc_stub.obj
 0001:00007850       AsrcGetInputBufStatus      10008850 f   asrcbase_mx25_topaz_v1_stub:mx25asrc_stub.obj
 0001:00007858       AsrcClosePair              10008858 f   asrcbase_mx25_topaz_v1_stub:mx25asrc_stub.obj
 0001:0000785c       AsrcSetP2PDeviceWML        1000885c f   asrcbase_mx25_topaz_v1_stub:mx25asrc_stub.obj
 0001:00007864       AsrcConfigPair             10008864 f   asrcbase_mx25_topaz_v1_stub:mx25asrc_stub.obj
 0001:0000786c       AsrcSetOutputBuf           1000886c f   asrcbase_mx25_topaz_v1_stub:mx25asrc_stub.obj
 0001:00007880       AsrcSetInputBuf            10008880 f   asrcbase_mx25_topaz_v1_stub:mx25asrc_stub.obj
 0001:00007894       GetLastError               10008894 f   coredll:COREDLL.dll
 0001:000078a4       CloseHandle                100088a4 f   coredll:COREDLL.dll
 0001:000078b4       Sleep                      100088b4 f   coredll:COREDLL.dll
 0001:000078c4       RegCloseKey                100088c4 f   coredll:COREDLL.dll
 0001:000078d4       RegQueryValueExW           100088d4 f   coredll:COREDLL.dll
 0001:000078e4       RegOpenKeyExW              100088e4 f   coredll:COREDLL.dll
 0001:000078f4       EnterCriticalSection       100088f4 f   coredll:COREDLL.dll
 0001:00007904       LeaveCriticalSection       10008904 f   coredll:COREDLL.dll
 0001:00007914       DisableThreadLibraryCalls  10008914 f   coredll:COREDLL.dll
 0001:00007924       SetLastError               10008924 f   coredll:COREDLL.dll
 0001:00007934       CeGetCallerTrust           10008934 f   coredll:COREDLL.dll
 0001:00007944       EventModify                10008944 f   coredll:COREDLL.dll
 0001:00007954       KernelIoControl            10008954 f   coredll:COREDLL.dll
 0001:00007964       WaitForMultipleObjects     10008964 f   coredll:COREDLL.dll
 0001:00007974       OpenDeviceKey              10008974 f   coredll:COREDLL.dll
 0001:00007984       InitializeCriticalSection  10008984 f   coredll:COREDLL.dll
 0001:00007994       CreateThread               10008994 f   coredll:COREDLL.dll
 0001:000079a4       CreateEventW               100089a4 f   coredll:COREDLL.dll
 0001:000079b4       WaitForSingleObject        100089b4 f   coredll:COREDLL.dll
 0001:000079c4       CeSetThreadPriority        100089c4 f   coredll:COREDLL.dll
 0001:000079d4       InterruptInitialize        100089d4 f   coredll:COREDLL.dll
 0001:000079e4       CeSafeCopyMemory           100089e4 f   coredll:COREDLL.dll
 0001:000079f4       LocalAlloc                 100089f4 f   coredll:COREDLL.dll
 0001:00007a04       LocalFree                  10008a04 f   coredll:COREDLL.dll
 0001:00007a14       HalAllocateCommonBuffer    10008a14 f   ceddk:CEDDK.dll
 0001:00007a24       HalFreeCommonBuffer        10008a24 f   ceddk:CEDDK.dll
 0001:00007a34       MmUnmapIoSpace             10008a34 f   ceddk:CEDDK.dll
 0001:00007a44       MmMapIoSpace               10008a44 f   ceddk:CEDDK.dll
 0001:00007a54       DDKGpioWriteDataPin        10008a54 f   cspddk:CSPDDK.dll
 0001:00007a64       DDKIomuxSetPinMux          10008a64 f   cspddk:CSPDDK.dll
 0001:00007a74       DDKClockSetGatingMode      10008a74 f   cspddk:CSPDDK.dll
 0001:00007a84       DDKSdmaAllocChain          10008a84 f   cspddk:CSPDDK.dll
 0001:00007a94       DDKSdmaOpenChan            10008a94 f   cspddk:CSPDDK.dll
 0001:00007aa4       DDKSdmaSetBufDesc          10008aa4 f   cspddk:CSPDDK.dll
 0001:00007ab4       DDKSdmaStopChan            10008ab4 f   cspddk:CSPDDK.dll
 0001:00007ac4       DDKSdmaStartChan           10008ac4 f   cspddk:CSPDDK.dll
 0001:00007ad4       DDKSdmaInitChain           10008ad4 f   cspddk:CSPDDK.dll
 0001:00007ae4       DDKSdmaClearBufDescStatus  10008ae4 f   cspddk:CSPDDK.dll
 0001:00007af4       DDKSdmaGetChainStatus      10008af4 f   cspddk:CSPDDK.dll
 0001:00007b04       timeSetEvent               10008b04 f   mmtimer:MMTimer.dll
 0001:00007b14       timeKillEvent              10008b14 f   mmtimer:MMTimer.dll
 0001:00007b24       CSPIOpenHandle             10008b24 f   spisdk_common_topaz_v1:spisdk.obj
 0001:00007b64       CSPIExchange               10008b64 f   spisdk_common_topaz_v1:spisdk.obj
 0001:00007bac       DllEntry                   10008bac f   spisdk_common_topaz_v1:spisdk.obj
 0001:00007bc0       I2CCloseHandle             10008bc0 f   i2csdk:I2CSDK.dll
 0001:00007bd0       I2CSetMasterMode           10008bd0 f   i2csdk:I2CSDK.dll
 0001:00007be0       I2COpenHandle              10008be0 f   i2csdk:I2CSDK.dll
 0001:00007bf0       I2CTransfer                10008bf0 f   i2csdk:I2CSDK.dll
 0001:00007c00       ??2@YAPAXI@Z               10008c00 f   corelib1:COREDLL.dll
 0001:00007c10       ??3@YAXPAX@Z               10008c10 f   corelib1:COREDLL.dll
 0001:00007c20       __C_specific_handler       10008c20 f   corelib1:COREDLL.dll
 0001:00007c30       memcpy                     10008c30 f   corelib1:COREDLL.dll
 0001:00007c40       memset                     10008c40 f   corelib1:COREDLL.dll
 0001:00007c50       memcmp                     10008c50 f   corelib1:COREDLL.dll
 0001:00007c60       _purecall                  10008c60 f   corelib1:COREDLL.dll
 0001:00007c70       __rt_sdiv64by64            10008c70 f   corelib1:COREDLL.dll
 0001:00007c80       __rt_udiv                  10008c80 f   corelib1:COREDLL.dll
 0001:00007c90       wcscpy                     10008c90 f   corelib1:COREDLL.dll
 0001:00007ca0       CreateFileW                10008ca0 f   coredll:COREDLL.dll
 0001:00007cb0       DeviceIoControl            10008cb0 f   coredll:COREDLL.dll
 0001:00007cfc       __IMPORT_DESCRIPTOR_COREDLL 10008cfc     coredll:COREDLL.dll
 0001:00007d10       __IMPORT_DESCRIPTOR_CEDDK  10008d10     ceddk:CEDDK.dll
 0001:00007d24       __IMPORT_DESCRIPTOR_CSPDDK 10008d24     cspddk:CSPDDK.dll
 0001:00007d38       __IMPORT_DESCRIPTOR_MMTimer 10008d38     mmtimer:MMTimer.dll
 0001:00007d4c       __IMPORT_DESCRIPTOR_I2CSDK 10008d4c     i2csdk:I2CSDK.dll
 0001:00007d60       __NULL_IMPORT_DESCRIPTOR   10008d60     coredll:COREDLL.dll
 0002:00000000       __imp_MmUnmapIoSpace       1000a000     ceddk:CEDDK.dll
 0002:00000004       __imp_HalFreeCommonBuffer  1000a004     ceddk:CEDDK.dll
 0002:00000008       __imp_HalAllocateCommonBuffer 1000a008     ceddk:CEDDK.dll
 0002:0000000c       __imp_MmMapIoSpace         1000a00c     ceddk:CEDDK.dll
 0002:00000010       \177CEDDK_NULL_THUNK_DATA  1000a010     ceddk:CEDDK.dll
 0002:00000014       __imp_RegOpenKeyExW        1000a014     coredll:COREDLL.dll
 0002:00000018       __imp_EnterCriticalSection 1000a018     coredll:COREDLL.dll
 0002:0000001c       __imp_LeaveCriticalSection 1000a01c     coredll:COREDLL.dll
 0002:00000020       __imp_DisableThreadLibraryCalls 1000a020     coredll:COREDLL.dll
 0002:00000024       __imp_SetLastError         1000a024     coredll:COREDLL.dll
 0002:00000028       __imp_CeGetCallerTrust     1000a028     coredll:COREDLL.dll
 0002:0000002c       __imp_EventModify          1000a02c     coredll:COREDLL.dll
 0002:00000030       __imp_KernelIoControl      1000a030     coredll:COREDLL.dll
 0002:00000034       __imp_WaitForMultipleObjects 1000a034     coredll:COREDLL.dll
 0002:00000038       __imp_RegQueryValueExW     1000a038     coredll:COREDLL.dll
 0002:0000003c       __imp_InitializeCriticalSection 1000a03c     coredll:COREDLL.dll
 0002:00000040       __imp_CreateThread         1000a040     coredll:COREDLL.dll
 0002:00000044       __imp_CreateEventW         1000a044     coredll:COREDLL.dll
 0002:00000048       __imp_WaitForSingleObject  1000a048     coredll:COREDLL.dll
 0002:0000004c       __imp_CeSetThreadPriority  1000a04c     coredll:COREDLL.dll
 0002:00000050       __imp_InterruptInitialize  1000a050     coredll:COREDLL.dll
 0002:00000054       __imp_CeSafeCopyMemory     1000a054     coredll:COREDLL.dll
 0002:00000058       __imp_LocalAlloc           1000a058     coredll:COREDLL.dll
 0002:0000005c       __imp_LocalFree            1000a05c     coredll:COREDLL.dll
 0002:00000060       __imp_RegCloseKey          1000a060     coredll:COREDLL.dll
 0002:00000064       __imp_Sleep                1000a064     coredll:COREDLL.dll
 0002:00000068       __imp_CloseHandle          1000a068     coredll:COREDLL.dll
 0002:0000006c       __imp_OpenDeviceKey        1000a06c     coredll:COREDLL.dll
 0002:00000070       __imp_GetLastError         1000a070     coredll:COREDLL.dll
 0002:00000074       __imp_DeviceIoControl      1000a074     coredll:COREDLL.dll
 0002:00000078       __imp_CreateFileW          1000a078     coredll:COREDLL.dll
 0002:0000007c       __imp_wcscpy               1000a07c     corelib1:COREDLL.dll
 0002:00000080       __imp___rt_udiv            1000a080     corelib1:COREDLL.dll
 0002:00000084       __imp___rt_sdiv64by64      1000a084     corelib1:COREDLL.dll
 0002:00000088       __imp__purecall            1000a088     corelib1:COREDLL.dll
 0002:0000008c       __imp_memcmp               1000a08c     corelib1:COREDLL.dll
 0002:00000090       __imp_memset               1000a090     corelib1:COREDLL.dll
 0002:00000094       __imp_memcpy               1000a094     corelib1:COREDLL.dll
 0002:00000098       __imp___C_specific_handler 1000a098     corelib1:COREDLL.dll
 0002:0000009c       __imp_??3@YAXPAX@Z         1000a09c     corelib1:COREDLL.dll
 0002:000000a0       __imp_??2@YAPAXI@Z         1000a0a0     corelib1:COREDLL.dll
 0002:000000a4       \177COREDLL_NULL_THUNK_DATA 1000a0a4     coredll:COREDLL.dll
 0002:000000a8       __imp_DDKSdmaClearBufDescStatus 1000a0a8     cspddk:CSPDDK.dll
 0002:000000ac       __imp_DDKIomuxSetPinMux    1000a0ac     cspddk:CSPDDK.dll
 0002:000000b0       __imp_DDKClockSetGatingMode 1000a0b0     cspddk:CSPDDK.dll
 0002:000000b4       __imp_DDKSdmaAllocChain    1000a0b4     cspddk:CSPDDK.dll
 0002:000000b8       __imp_DDKSdmaOpenChan      1000a0b8     cspddk:CSPDDK.dll
 0002:000000bc       __imp_DDKSdmaSetBufDesc    1000a0bc     cspddk:CSPDDK.dll
 0002:000000c0       __imp_DDKSdmaStopChan      1000a0c0     cspddk:CSPDDK.dll
 0002:000000c4       __imp_DDKSdmaStartChan     1000a0c4     cspddk:CSPDDK.dll
 0002:000000c8       __imp_DDKSdmaGetChainStatus 1000a0c8     cspddk:CSPDDK.dll
 0002:000000cc       __imp_DDKGpioWriteDataPin  1000a0cc     cspddk:CSPDDK.dll
 0002:000000d0       __imp_DDKSdmaInitChain     1000a0d0     cspddk:CSPDDK.dll
 0002:000000d4       \177CSPDDK_NULL_THUNK_DATA 1000a0d4     cspddk:CSPDDK.dll
 0002:000000d8       __imp_I2CTransfer          1000a0d8     i2csdk:I2CSDK.dll
 0002:000000dc       __imp_I2COpenHandle        1000a0dc     i2csdk:I2CSDK.dll
 0002:000000e0       __imp_I2CSetMasterMode     1000a0e0     i2csdk:I2CSDK.dll
 0002:000000e4       __imp_I2CCloseHandle       1000a0e4     i2csdk:I2CSDK.dll
 0002:000000e8       \177I2CSDK_NULL_THUNK_DATA 1000a0e8     i2csdk:I2CSDK.dll
 0002:000000ec       __imp_timeKillEvent        1000a0ec     mmtimer:MMTimer.dll
 0002:000000f0       __imp_timeSetEvent         1000a0f0     mmtimer:MMTimer.dll
 0002:000000f4       \177MMTimer_NULL_THUNK_DATA 1000a0f4     mmtimer:MMTimer.dll
 0002:00000108       ?szNames@?1??GetListText@MixerControlInputMux@@QAAXPAUtMIXERCONTROLDETAILS_LISTTEXT@@K@Z@4PAPBGA 1000a108     esai_common_topaz_v1:mixerdrv.obj
 0002:00000118       ?g_pHWContext@@3PAVHardwareContext@@A 1000a118     esai_common_topaz_v1:hwctxt.obj

 entry point at        0001:00007bac

 Static symbols

